:100000006E28FF3FFF3FFF3F0E3003138312FA00BD
:10001000FA0B082800000800031383129F01C03068
:100020009F04403083161F04F00070089F0080304A
:1000300070049F0083122408F000F00D7010F00D82
:100040007010F00D701070089F041F1404201F150D
:1000500000301F190130F2007208013A031D3228E6
:10006000000028281E08F200F3017208F300F201D4
:100070007208A5007308A60083161E087204831276
:10008000A5007308A6000030A6041F102508F00084
:100090002608F10008000030031383169818013079
:1000A000F1007108003A031D572800004B28831205
:1000B00024089900080003138316981690308312C1
:1000C0009800831606158612003083128C1A0130B0
:1000D000F1007108013A0319642808007030031315
:1000E00083168F0000300F190130F2007208003AB9
:1000F00003197228043085008601831285010130BE
:100100008600043083169B0040309F0033309900F6
:1001100018155B200230A4000C207008A0007108A4
:10012000A1000230F400740803199B28F10CF00CB4
:10013000F113FF3F94287008A0007108A100700817
:10014000A2007108A3007008A4004B20D030FB006F
:10015000FF30FA00FB0BAD28B028FA0BAD28AA2817
:100160003F30FA00FA0BB228000000008A28B728B6
:04400E00FC3FFFFF75
:00000001FF
